:1000000019C0A4C118C21895189518951895189577
:100010001895189518951895189518951895189578
:100020001895189518951895189518951895189568
:10003000189518958FEF8DBFC0EEE8ED4E2E82E03B
:100040008EBFD2E0F2E05F2EEEEFF1E0A0E0B1E093
:10005000A89584B7082E877F84BF88E1992780936D
:1000600060009093600088278D933197E9F76624AC
:100070008FEF84B9389A399A3A9A3B9A519A80917B
:1000800069008C7F826080936900E89A80916900A2
:10009000837F886080936900E99A80E085B980E079
:1000A00088B95998F89448D410ED5DD410E05BD429
:1000B00051D442D411ED57D475D4A3E0B1E01C93D0
:1000C00071D4A2E0B1E01C936BD4A1E0B1E01C9329
:1000D000A1E0B1E08C918F738C93A1E0B1E09C9191
:1000E00037D3A1E0B1E08C93A2E0B1E09C9130D392
:1000F000A2E0B1E08C937894009102014AE0F7D33A
:10010000AEE0B1E00C9300910E014AE0049FA0E044
:10011000B1E00C920091020140910001041BADE09E
:10012000B1E00C93009101014AE0E1D3A0E1B1E01C
:100130000C93009110014AE0049FA0E0B1E00C9202
:100140000091010140910001041BAFE0B1E00C936C
:1001500084E18093140182E090E0A7E1B1E08D9307
:100160009C93E2D184E18093140181E090E0A7E1C7
:10017000B1E08D939C93D8D184E18093140180E009
:1001800090E0A7E1B1E08D939C93CED18FEF809367
:1001900014018FEF9FEFA7E1B1E08D939C93C4D141
:1001A00084E18093140180E090E0A7E1B1E08D93B9
:1001B0009C93BAD184E18093140181E090E0A7E19F
:1001C000B1E08D939C93B0D184E18093140182E0DF
:1001D00090E0A7E1B1E08D939C93A6D1F894599A51
:1001E00080E0E9E2FCD26CEC80E0E9E2BB27A6E12A
:1001F00021E02A9320D364E480E0E9E2BB27A6E172
:1002000021E02A9318D38EEE92E0B2D2599880E082
:10021000E9E2E5D26CEC80E0E9E2BB27A6E121E06F
:100220002A9309D36EEB80E0E9E2BB27A6E121E047
:100230002A9301D380E0A4E0B1E0E9E229E02A9327
:1002400034D388E0E4E0F1E062D3402F00910C0168
:10025000041709F015C0A5E0B1E09C91A4E0B1E05D
:100260008C91A5E1B1E08D939C93A5E1B1E00D9156
:100270001C9140E150E021D2A5E1B1E04D935C93A7
:100280007894009115014AE032D3A0E1B1E00C93DB
:10029000009110014AE0049FA0E0B1E00C920091AF
:1002A000150140910001041BAFE0B1E00C938BE01D
:1002B00080930E018CE080930D0184E18093140102
:1002C0008CEF9FEFA7E1B1E08D939C932DD184E15A
:1002D000809314018DEF9FEFA7E1B1E08D939C9384
:1002E00023D184E1809314018EEF9FEFA7E1B1E069
:1002F0008D939C9319D18FEF809314018FEF9FEF13
:10030000A7E1B1E08D939C930FD184E18093140118
:100310008EEF9FEFA7E1B1E08D939C9305D184E12F
:10032000809314018DEF9FEFA7E1B1E08D939C9333
:10033000FBD084E1809314018CEF9FEFA7E1B1E043
:100340008D939C93F1D0AECEF894FFCF0F921F9275
:100350002F923F924F925F927F92AF92BF920F93F4
:100360001F932F933F934F935F936F937F938F933D
:100370009F93AF93BF93CF93DF93EF93FF938FB789
:100380008F93A1E0B1E08C918F5F8C93009101017C
:10039000073110F009F001C003C080E08093010133
:1003A000009101014AE0A3D2A0E1B1E00C930091D9
:1003B00010014AE0049FA0E0B1E00C92009101011D
:1003C00040910001041BAFE0B1E00C93A1E0B1E06B
:1003D0008C91B8D1A0E0B1E08C93809100018F7B2B
:1003E00080930001A9D210EDBED212E0BCD2A0E0F1
:1003F000B1E01C91B8D2AED288EC90E0B9D18F9127
:100400008FBFFF91EF91DF91CF91BF91AF919F91FE
:100410008F917F916F915F914F913F912F911F919C
:100420000F91BF90AF907F905F904F903F902F9033
:100430001F900F9018950F921F922F923F924F92FC
:100440005F927F92AF92BF920F931F932F933F9330
:100450004F935F936F937F938F939F93AF93BF93CC
:10046000CF93DF93EF93FF938FB78F93A2E0B1E029
:100470008C918F5F8C93009102010B3310F009F087
:1004800001C003C080E080930201009102014AE0B4
:100490002ED2AEE0B1E00C9300910E014AE0049F31
:1004A000A0E0B1E00C920091020140910001041B18
:1004B000ADE0B1E00C93A2E0B1E08C9143D1A0E0BB
:1004C000B1E08C9339D210ED4ED210E04CD210E056
:1004D0004AD240D231D210ED46D211E044D2A0E04F
:1004E000B1E01C9140D236D288EC90E041D18F919E
:1004F0008FBFFF91EF91DF91CF91BF91AF919F910E
:100500008F917F916F915F914F913F912F911F91AB
:100510000F91BF90AF907F905F904F903F902F9042
:100520001F900F901895089581E08093120100911B
:100530001201043010F009F042C0A0E0B1E0BA931B
:10054000AA935A924A92A2E1B1E0AD90BB24ACE0EA
:10055000B1E0AA0DBB1D8C91A42DB52D8C9381E02B
:10056000A5D03DD0249681E09DD0A0E0B1E08C9153
:1005700085B90091120140911701040FA3E1B1E088
:100580000C93A3E1B1E08C91A8E2B0E00AD1FFD0D6
:100590009C91982B9C9385E090E0EAD0A3E1B1E098
:1005A0008C91A8E2B0E0FDD0F2D08C9189238C939D
:1005B000A2E1B1E08C918F5F8C9308F4B8CFA1E1F8
:1005C000B1E08C918F5F8C934091140100911101E7
:1005D000041709F0A9CF80E0809311010895A88144
:1005E000B9810C91013009F005C08CE7AA81BB816B
:1005F0008C9357C0023009F005C082E1AA81BB810B
:100600008C934FC0033009F005C088E1AA81BB81FB
:100610008C9347C0043009F005C08CE2AA81BB81ED
:100620008C933FC0053009F005C089E0AA81BB81E9
:100630008C9337C0063009F005C081E0AA81BB81E8
:100640008C932FC0073009F005C088E7AA81BB81D1
:100650008C9327C0083009F005C080E0AA81BB81D7
:100660008C931FC0093009F005C088E0AA81BB81C6
:100670008C9317C0003009F005C080E4AA81BB81CB
:100680008C930FC00B3009F005C08AE2AA81BB81B0
:100690008C9307C00C3009F004C083E4AA81BB81AD
:1006A0008C930895481A8827580A0895480E882779
:1006B000581E089500FC10D0089503D01ED001F8F4
:1006C000F9CF0024E89457FF02C009D0689400F8DD
:1006D0000BD010F80124089502D009D00895509548
:1006E00040954F5F5F4F0895E89417FF0895009578
:1006F00010950F5F1F4F68940895352F242FE894AD
:10070000452B11F468940895512F402F002711278D
:1007100080E1440F551F001F111F021B130B416086
:1007200018F4020F131F4E7F8A9599F70895982F9A
:1007300082958F70805D8D939F70905D9D938827CB
:100740008C9308954AE0082FD2D00295802B08950B
:10075000892F8F70905110F0865FFCCF08953197EC
:10076000F1F70895689462F80895E89462F808959E
:10077000EF93FF93EE27E82BE92B31F0E0EDF7E064
:100780003197F1F70197D1F7FF91EF91089591E03B
:10079000882321F08894991F8A95E9F7892F9095ED
:1007A0000895883018F011968850FBCF0895018184
:1007B000082B01831281192312830000000000001E
:1007C0000000000000000000000000000000000029
:1007D0000000000000000000000000000895C2DFDB
:1007E000FF27D5DFE4DFEF93FF93ECEBF3E0B7DF18
:1007F000FF91EF91182B128309230183EF93FF934D
:10080000E0EBF0E0ACDFFF91EF911081182359F499
:10081000EF93FF93ECEBF3E0A2DFFF91EF911081F8
:10082000182309F0A2DFEF93FF93ECEBF3E097DFDF
:10083000FF91EF910895ABDFFF2729915D9148E08B
:10084000B6DF000000000000000000000000000013
:100850000000000000000000000000000000000098
:1008600000000000579510F4182B1283EF93FF93AC
:10087000E4E7F0E074DFFF91EF91182B12830000A2
:100880000000000000000000000000000000000068
:100890000000000000000000000000000000000058
:1008A0004A9571F62A9551F6089571DFFF2729912F
:1008B00048E055277CDF09230183EF93FF93E8E0AD
:1008C000F0E04DDFFF91EF9188941081182309F03B
:1008D00008945795EF93FF93E6E5F0E040DFFF9132
:1008E000EF914A9539F75D932A9511F70895FF9393
:1008F000881BF9E0001FFA9511F4FF910895881FF5
:10090000841B18F4840F8894F5CF0894F3CF002744
:100910006CE8719198E00695779577FF18F477FD6C
:1009200008F006279A95B9F78A9599F7089544989B
:1009300045983C983D9808953D9A3C9803D03D9841
:1009400001D03C9AEF93FF93E6E0F0E008DFFF91DF
:10095000EF9108953D9A3C9AF5DF3D98359BFECF87
:10096000F1DF3C98EFCF0894111F01C0110F69F01F
:100970003D9A18F400003C9802C03C9A00C0E2DFA7
:100980003D98359BFECFDEDFF1CF3D9A3C98DADF14
:100990003D98359BFECFE8943499689462F8D2CFA5
:1009A000089401C08894331F11E03D9A3C98CADF37
:1009B0003D98359BFECFC6DF889434990894111F6B
:1009C000A0F73D9A379510F43C9801C03C9ABADFE5
:0A09D0003D98359BFECFB6DF089579
:00000001FF
